:040000000207B93208
:01000B0032C2
:0100130032BA
:01001B0032B2
:0100230032AA
:01002B0032A2
:0B07B9007581331200A0E5826003028E
:0207C400002C07
:0807C6007900E94400601B7A90
:0507CE00009008017815
:0C07D3000075A000E493F2A308B8000237
:0907DF0005A0D9F4DAF275A0FFBF
:0807E8007800E84400600C7980
:0D07F00000900000E4F0A3D8FCD9FAF6D880
:0107FD00FDFE
:0307FE0002002CCA
:05002C0012006380FEDC
:0E003100AA82AB8375C8308A048CCA8B027B0E
:0E003F00008ACB8CCC8ACDD2CA759850D2994B
:01004D002290
:02004E00AA8284
:0500500010990280FB85
:020055008A9986
:010057002286
:0500580010980280FB7E
:05005D00E59985998280
:01006200227B
:0E00630090FFBF12003174BFC0E074FFC0E018
:0C0071007495C0E07400C0E07402C0E0B0
:09007D001200A4E58124FBF581C9
:0E008600120058E5822401F58212004E80F22D
:010094002249
:0B00950048656C6C6F212025640A0098
:0300A00075820066
:0100A300223A
:0600A400C032858132E547
:0600AA003224FBF531E5F4
:0D00B0003224FBF886820886830886F01251
:0800BD0006E3AA82AB838B83EA
:0600C500853281D03222D9
:0600CB00C032858132E520
:0600D1003224F8F530E5D1
:0800D7003224F8F8862D08869A
:0500DF002E08862FE54C
:0D00E4003224FBF886820886830886F0121D
:0800F10001C3AA82AB838B83DB
:0600F900853281D03222A5
:0800FF00C032858132AA823073
:02010700001ADC
:05010900AB22AC23ADA8
:0C010E00248B828C838DF0EA12071F0501
:06011A0022E4B5220905F4
:0101200023BB
:02012100800557
:050123008A8212004E6B
:07012800052BE4B52B0205D5
:01012F002CA3
:06013000853281D032226D
:0C013600C032858132AA82C374099AB3DA
:05014200E433FB600640
:0601470074302AFB800F5A
:03014D0030010678
:0601500074572AFC800434
:0401560074372AFCD4
:02015A008C0314
:05015C008B821200FF80
:06016100853281D032223C
:0C016700C032858132E582FAC4540FF5E5
:0E01730082C002120136D002740F5AF58212B9
:02018100013645
:06018300853281D032221A
:020189007A20DA
:05018B00BA0002803201
:07019000C3E52533F525E569
:050197002633F526E50A
:05019C002733F527E503
:0501A1002833F528E5FC
:0601A6002933F529C3E531
:0501AC0029952A400E18
:0601B100E529C3952AF5C3
:0701B70029AB2574012BF5B3
:0101BE00251B
:0301BF001A80C9DA
:0101C200221A
:0C01C300AA82AB83ACF0E4F52CF52B8A8B
:0401CF00228B238CD0
:0601D30024EA4B4C70040D
:0401D900C2008002DE
:0201DD00D2004E
:0501DF00AA2DAB2EACBF
:0D01E4002F8A828B838CF012078DFD740131
:0801F1002AF52DE43BF52E8CEC
:0901F9002F8D02ED70030206C512
:05020200BA2502800393
:030207000206BD2F
:05020A00C203C204C2A2
:04020F0005C206C25C
:0502130007752A00C27E
:0402180008C209C24D
:08021C000A7B007CFFAD2DAE52
:030224002EAF2FCB
:0E0227008D828E838FF012078DFAA3AD82AE0A
:06023500838D2D8E2E8F3B
:04023B002FBA2507AA
:07023F008A821200FF809982
:0E0246008A82C002C003C004C005C006C00703
:0E02540012070AE582D007D006D005D004D0EC
:0502620003D002602240
:03026700BCFF12C7
:0E026A00EB75F00AA4F8EA24D028FBBB00AF25
:04027800D20480AB81
:0D027C00EC75F00AA4F8EA24D028FC809E5E
:03028900BA2E0486
:04028C007C008097DB
:0E0290008A82C002C003C004C005C006C007B9
:0D029E00120750E58224FF9201D007D00620
:0B02AB00D005D004D003D002300103C6
:0302B6005302DF11
:0502B900BA200280558F
:0502BE00BA2B02804B89
:0502C300BA2D0280418C
:0502C800BA4202804B68
:0502CD00BA430280505D
:0602D200BA4403020467B8
:0602D800BA460302047D9A
:0602DE00BA4903020467A7
:0502E400BA4C02803459
:0602E900BA4F0302046E8F
:0602EF00BA50030203F502
:0502F500BA5302804134
:0602FA00BA550302047373
:06030000BA580302047864
:030306000204816D
:05030900D203020227EF
:05030E00D205020227E8
:05031300D206020227E2
:05031800D208020227DB
:05031D00D209020227D5
:0C032200E53024FEF888308604088605CB
:0D032E00188C82C0031200FFD00302048A65
:0C033B00E53024FDF888308604088605B3
:0A03470008860618188C258D268EF6
:0D035100278C828D838EF0C003120765ACEF
:0A035E0082AD83D0038C022003253A
:05036800C3EA9B5020D8
:06036D00EBC39AFB8B05B7
:0A0373008D061D8D03BE00028010F0
:0E037D00758220C002C0051200FFD005D0021C
:02038B0080E60A
:07038D00852582852683858A
:0803940027F012078DFD602E19
:05039C00AD25AE26AF07
:0C03A1002774012DF8E43EF98F04882534
:0B03AD0089268C278D828E838FF01232
:0E03B800078DFDF582C002C0031200FFD003C6
:0403C600D00280C31E
:0603CA0020030302048A77
:0803D000C3EA9B400302048A0A
:0603D800EBC39AFB8B044D
:0B03DE008C051C8C03BD000302048A88
:0C03E900758220C0041200FFD00480E9DF
:0C03F500E53024FDF888308604088605F9
:0A04010008860618188C258D268E3B
:08040B0027C374039527500478
:040413007C048002E3
:02041700AC2710
:0E041900EC9006F993FCF582C0031200FFD0B0
:0E0427000375823AC0031200FFD003758230C5
:0D043500C0031200FFD003758278C00312CF
:0804420000FFD003E527601163
:07044A00E527B40302800A5C
:0A045100852682C003120167D00364
:0C045B00852582C003120167D0038023B6
:07046700D207752A0A801C70
:05046E00752A0880174B
:05047300752A0A801249
:05047800752A10800D43
:04047D00D20A800916
:090481008A82C0031200FFD003BF
:03048A00300A53E2
:0C048D00E53024FCF88830860408860561
:0C0499000886060886071818188C258DA8
:0404A500268E278FE9
:0304A9002875258E
:0304AC00FF7526B3
:0404AF0006752702A5
:0504B300AC25AD26AEF2
:0C04B8002774012CFFE43DF88E018F2515
:0B04C400882689278C828D838EF01221
:0A04CF00078DFC8C0270030201DFB0
:0704D9008A821200FF80D3AC
:0704E000E52A70030201DFB1
:0304E700300825B5
:0C04EA00E53014F888308604EC3395E00F
:0804F600FDFEFF8C258D268E12
:0404FE00278F2820FC
:0205020007519F
:070504007526007527007544
:04050B0028008046FE
:03050F0030091F91
:0C051200E53024FCF888308604088605DB
:0C051E000886060886071818188C258D22
:04052A00268E278F63
:03052E00288024FE
:0C053100E53024FEF888308604088605BA
:0C053D0018ED3395E0FEFF8C258D268E16
:04054900278F2820B0
:02054D0007069F
:06054F007527007528006D
:030555003007224A
:05055800E52830E71B5F
:0B055D00C3E49525FCE49526FDE49521
:0705680027FEE49528FF8C3B
:04056F00258D268E22
:05057300278F28800223
:02057800C207B8
:04057A00D2027C002D
:0D057E00752900C003C004120189D004D00B
:0C058B000320020BD0F0E529C442F0C0B0
:03059700F08004ED
:04059A00E529C0E0AF
:07059E000CB202E52560022A
:0205A50080D7FD
:0405A700E5266002E3
:0205AB0080D1FD
:0405AD00E5276002DC
:0205B10080CBFD
:0805B300E528700474018001C9
:0105BB00E45B
:0505BC00FD8C0260BD92
:0305C100BB00027A
:0205C4007B01B9
:0305C600200437D7
:0305C900200334D8
:0205CC008B049E
:0905CE008A057E000DBD00010E3E
:0E05D7008C077800C3ED9FEE648088F063F01F
:0A05E5008095F0E433FD8C036011F3
:0E05EF00758220C002C0041200FFD004D002AA
:0305FD001C80CE91
:03060000300711AF
:0E06030075822DC002C0031200FFD003D0028A
:030611001B802B20
:05061400BA000280267F
:0306190030051198
:0E061C0075822BC002C0031200FFD003D00273
:03062A001B801220
:03062D0030060F85
:0E063000758220C002C0031200FFD003D0026A
:01063E001BA0
:03063F0020032471
:020642008B0427
:0A0644008C051C8C03C3EA9D5025B1
:03064E0030040471
:040651007D30800276
:020655007D2006
:0E0657008D82C002C0041200FFD004D00280C9
:01066500DEB6
:05066600C3EA9B5006F1
:06066B00EBC39AFB8002C4
:020671007B000C
:020673008A04F7
:060675008C051CED602560
:0C067B00B20220020AD0E000C0E0C4542B
:030687000F8004DD
:04068A00D0E0540F59
:0A068E00F529852982C003C004127B
:080698000136D004D00380D527
:0606A0002003030201DF4C
:0B06A6008B041BC3E49C40030201DF37
:0C06B100758220C0031200FFD00380E916
:0806BD008A821200FF0201DF36
:0306C500300014EE
:0D06C8007582001200FFE52B24FFF582E58E
:0706D5002C34FFF5838006C1
:0606DC00852B82852C83B2
:0106E20022F5
:0806E30085822D85832E85F030
:0306EB002F853127
:0A06EE003090000075F0001201C307
:0106F80022DF
:0606F900495843502D009A
:0B06FF003C4E4F20464C4F41543E0043
:05070A00AA82BA3000D4
:02070F00400A9E
:06071100C374399A400494
:0407170075820122C4
:03071B00758200E4
:01071E0022B8
:0E071F00C0E0E5F0601114601914600714606A
:05072D00181414600423
:04073200D0E080197A
:0B073600D0E0C000A882F6D000800ECA
:05074100D0E0F080098A
:09074600D0E0C000A882F2D0004E
:01074F002287
:05075000AA82BA61005D
:02075500400A58
:06075700C3747A9A40040D
:04075D00758201227E
:030761007582009E
:010764002272
:0A076500AA82AB83ACF07D007E0099
:0E076F008A828B838CF012078DFFA3AA82ABC7
:04077D0083EF60079F
:070781000DBD00EA0E80E748
:040788008D828E834D
:01078C00224A
:0E078D00E5F060111460171460171460171463
:07079B0014600474FF8016D6
:0907A200C000A882E6D000800D21
:0307AB00E0800AE1
:0307AE009380072E
:0707B100C000A882E2D000A5
:0107B800221E
:00000001FF
